:100000000C9411060C9453280C9480280C943906F7
:100010000C9439060C94870C0C9439060C94390610
:100020000C9439060C9439060C9439060C94390654
:100030000C9439060C9439060C9439060C94390644
:100040000C94AD280C9439060C94452C0C94802CFF
:100050000C9439060C9439060C9439060C94390624
:100060000C9439060C943906BC1BC31BC31BBC1B68
:10007000C31BC31BC31BC31BC31BC31BC31BC31B90
:10008000C31BC31BC31BC31BC31B311BC31BC31B12
:10009000C31BC31BC31B941AC31BC31BC31BC31BA0
:1000A000C31BC31BC31BC31BC31BC31BC31BC31B60
:1000B000C31BC31BC31B3D1B3D1B3D1B3D1B3D1BEE
:1000C0003D1B3D1B3D1B3D1BC31BC31BC31BC31B58
:1000D000C31BC31B991A3C1B3C1B3C1B3C1BC31B77
:1000E0004D1B551B5D1B651B6D1B751B7D1B851BF0
:1000F0008F1B991BA31BAD1BE01AA01AC31BC31BAC
:10010000C31BC31B311BC31BC31BC31BC31BC31B91
:10011000C31BC31BC31B3B1B3B1B3B1B3B1BC31B0F
:100120004D1B551B5D1B651B6D1B751B7D1B851BAF
:100130008F1B991BA31BAD1BE01AA01AC31BC31B6B
:10014000C31BC31B311BF41BF41BF41BF41BF41B5C
:10015000F41BF41BF41BF41BF41BF41BF41BF41B27
:10016000151D151D151D151D151D151D3B1C451CAB
:100170004F1C591CBF1CC91CD71CE91C861DF61D31
:10018000C71DCC1DD11DD61DDB1DE01DE51DF61DB7
:10019000F01DEF2404251025192526254C2554256E
:1001A00077256425456E746572206D656E752E2EFB
:1001B0002E00546F67676C6564206D6963726F50C1
:1001C000504D00546F67676C656420696E76657288
:1001D0007465642050504D2100546F67676C6564EE
:1001E000205458206D7574696E672100546F6767DD
:1001F0006C65642074656C656D657472792100505E
:10020000726F746F636F6C206572726F72207769A2
:1002100074682052580054696D656F757420776852
:10022000656E20636F6E6E656374696E6720746FB0
:1002300020525800507265737320616E79206B658F
:100240007920746F2063616E63656C00436F6E6E1E
:10025000656374696E6720746F2052582C20706F2C
:100260007765722075702074686520525820287751
:100270006974682062696E6420706C7567206966B5
:10028000206E6F74207573696E6720616C77617979
:10029000732062696E642900546F67676C6564201F
:1002A00027696D6D656469617465206F757470751B
:1002B000742700546F67676C65642027736C6176E0
:1002C00065206D6F64652700546F67676C656420F7
:1002D00027616C776179732062696E642700546FBF
:1002E00067676C65642050504D206368616E6E6571
:1002F0006C206C696D6974005365742052535349C6
:1003000020696E6A656374696F6E206368616E6EE2
:10031000656C2028303D3D64697361626C6529001D
:100320005365742050504D206D696E696D756D2058
:1003300073796E630053657420626561636F6E202C
:10034000696E74657276616C0053657420626561D4
:10035000636F6E2064656C6179005365742062651B
:1003600061636F6E206672657175656E6379206971
:100370006E20487A3A20303D64697361626C652C66
:100380002050783D504D52206368616E6E656C2040
:10039000782C2046783D465253206368616E6E6526
:1003A0006C2078005365742050574D2073746F7023
:1003B0002064656C61792028302064697361626C07
:1003C00065642C20312D323535203D3D20302E31D5
:1003D00073202D2035306D696E29005365742050CF
:1003E000504D2073746F702064656C6179202830E3
:1003F0002064697361626C65642C20312D3235355F
:10040000203D3D20302E3173202D2035306D696E1A
:100410002900536574206661696C736166652064A8
:10042000656C61792028302064697361626C656451
:100430002C20312D323535203D3D20302E3173209A
:100440002D2035306D696E29002A2A2A2A2A2A2A67
:100450002A2A2A2A2A2A2A2A2A2A2A2A2A2A2A2AFC
:100460002A2A2A2A2A2A0052582041636B656420CE
:100470002D2072657665727420737563636573737E
:1004800066756C21002A2A2A2A2A2A2A2A2A2A2A36
:100490002A2A2A2A2A2A2A2A2A2A2A2A2A2A2A2ABC
:1004A0002A2A002A2A2A2A2A2A2A2A2A2A2A2A2AD6
:1004B0002A2A2A2A2A2A2A2A2A2A2A2A2A2A2A2A9C
:1004C0000052582041636B6564202D207570646173
:1004D0007465207375636365737366756C21002A98
:1004E0002A2A2A2A2A2A2A2A2A2A2A2A2A2A2A2A6C
:1004F0002A2A2A2A2A2A2A2A2A2A2A2A0056616CE1
:1005000069642063686F69636573206172653A206E
:100510005B315D2D5B31365D20286368616E6E65F1
:100520006C20312D31362900536574206F7574703D
:10053000757420666F7220706F727420005B585D56
:100540002061626F7274206368616E6765732061F9
:100550006E64206578697420525820636F6E6669F6
:1005600067005B535D207361766520736574746901
:100570006E677320746F205258005B525D20726565
:10058000766572742052582073657474696E67734F
:1005900020746F2064656661756C747300557365B3
:1005A000206E756D62657273205B312D445D207421
:1005B0006F206564697420706F727473205B452DC1
:1005C000515D20666F722073657474696E67730085
:1005D000202D20726563656976657220636F6E6693
:1005E0006967757261746F722C207278207377203E
:1005F000000A0A6F70656E4C52536E672000536597
:10060000742073657269616C2062617564726174D3
:10061000653A200056616C69642063686F696365A0
:10062000733A2031202D20342B34202F2032202DDE
:100630002038202F2033202D20382B34202F203419
:10064000202D203132202F2035202D2031322B3407
:10065000202F2036202D203136005365742043682A
:10066000616E6E656C20636F6E6669673A20005339
:1006700065742044617461726174652028302D3284
:10068000293A200053657420486F70206368616EBA
:100690006E656C7320286D61782032342C20736570
:1006A0007061726174656420627920636F6D6D6141
:1006B00073292076616C69642076616C756573209E
:1006C000312D3235353A2000536574206368616EF0
:1006D0006E656C2073706163696E672028783130B5
:1006E0006B487A293A200053657420524620706F77
:1006F0007765722028302D37293A20005365742001
:100700005246206D616769632028686578292065F5
:100710002E672E20307844454144463030443A20FC
:10072000005365742062617365206672657175653A
:100730006E63792028696E20487A293A20005B5A36
:100740005D20656E74657220726563656976657299
:1007500020636F6E66696775726174696F6E20756C
:1007600074696C79005B465D20646973706C6179B3
:100770002061637475616C206672657175656E6366
:100780006965732075736564005B525D2063616CFD
:1007900063756C6174652072616E646F6D206B654A
:1007A0007920616E6420686F70206C697374005BDF
:1007B000495D207265696E697469616C697A65204A
:1007C00073657474696E677320746F20736B6574DE
:1007D00063682064656661756C7473005B585D20A6
:1007E000726576657274206368616E6765732061F7
:1007F0006E642065786974206D656E75005B535D6D
:1008000020736176652073657474696E67732074F4
:100810006F20454550524F4D20616E6420657869C8
:1008200074206D656E7500557365206E756D62651B
:100830007273205B302D395D20746F20656469749C
:1008400020706172616D657465727300202D205394
:10085000797374656D20636F6E6669677572617414
:10086000696F6E000A0A6F70656E4C52536E672096
:10087000005129204F7574707574206265666F721F
:1008800065206C696E6B20283D465329203A200074
:10089000502920536C617665206D6F646520286552
:1008A00078706572696D656E74616C293A20004FCD
:1008B000292054696D65642042494E4420617420AA
:1008C0007374617274757020203A20004E29205094
:1008D000504D206F7574707574206C696D69746506
:1008E0006420202020203A200044495341424C45B6
:1008F00044004D292050504D205253534920746FCD
:10090000206368616E6E656C202020203A20004CC8
:10091000292050504D206D696E696D756D20737979
:100920006E63202875732920203A200044495341E2
:10093000424C4544004B29204661696C73616665F1
:1009400020626561636F6E20696E74762E20283197
:100950002D32353573293A20004A29204661696CC9
:100960007361666520626561636F6E2064656C61AA
:10097000792028302D323535203D3E20313073200E
:100980002D203135306D696E293A200049292046E5
:1009900061696C7361666520626561636F6E206674
:1009A00072712E203A200048292050574D20737430
:1009B0006F702064656C6179202020202020203A0F
:1009C000200047292050504D2073746F70206465BB
:1009D0006C6179202020202020203A200046292008
:1009E0004661696C736166652064656C617920207D
:1009F00020202020203A200050574D206368616E4F
:100A00006E656C200066756E6374696F6E3A2000C7
:100A10002920706F727420004454462055484620A7
:100A200033322D6269742031306368004F70656E17
:100A30004C52536E675258206D696E6920342F36C0
:100A4000636800466C7974726F6E2F4F72616E67C7
:100A50006552582055484620386368005258207423
:100A60007970653A200044697361626C656400487E
:100A70007A00203D3D200043616C63756C617465B4
:100A800064207061636B657420696E746572766151
:100A90006C3A20004229204D6963726F20286861FA
:100AA0006C66292050504D202020203A00412920FA
:100AB000496E7665727465642050504D20696E20D1
:100AC000202020203A003029204D75746520627561
:100AD0007A7A657220286D6F73746C79293A0039BF
:100AE000292053657269616C20626175647261745A
:100AF000653A00736D617274506F72740046725380
:100B00006B79005472616E73706172656E7400442B
:100B1000697361626C65640038292054656C656D89
:100B2000657472793A202020202020200037292067
:100B30004368616E6E656C20636F6E6669673A200C
:100B40002000362920446174617261746520283068
:100B50002D32293A20202000352920486F7020634B
:100B600068616E6E656C733A202020202000342965
:100B7000204368616E6E656C2073706163696E6797
:100B80003A202000332920524620706F776572206A
:100B900028302D37293A20202000322920524620A3
:100BA0006D616769633A20202020202020202000EA
:100BB00031292042617365206672657175656E63C7
:100BC000793A2020200000000000240027002A009D
:100BD00000000000250028002B000000000023007A
:100BE000260029000404040404040404020202028E
:100BF00002020303030303030102040810204080E0
:100C0000010204081020010204081020000000075F
:100C100000020100000304060000000000000000C4
:100C2000282E11241FBECFEFD8E0DEBFCDBF13E0CA
:100C3000A0E0B1E0E2E9FEE502C005900D92A63920
:100C4000B107D9F716E0A6E9B3E001C01D92A734B9
:100C5000B107E1F71CE0C2E2DCE004C02297FE012C
:100C60000E94242FC032D107C9F70E946D2E0C9428
:100C7000472F0C940000A0E0B0E0E1E4F6E00C9413
:100C8000F32EEC01A880B980CA80DB80A114B104E6
:100C9000C104D10441F484E2A82E89EDB82E8BE57D
:100CA000C82E87E0D82EC601B5012DE133EF41E013
:100CB00050E00E94D02E27EA31E440E050E00E944C
:100CC0007C2E7B018C01C601B5012DE133EF41E0A3
:100CD00050E00E94D02ECA01B9012CEE34EF4FEF44
:100CE0005FEF0E947C2E6E0D7F1D801F911F97FF6E
:100CF00004C06150704080409048688379838A8343
:100D00009B839B01AC015F77B901CA01CDB7DEB708
:100D1000EAE00C940F2F0E943B06089581EB92E0CD
:100D20000E943B0608956093B1027093B2028093D3
:100D3000B3029093B4020895A0E0B0E0E2EAF6E0D6
:100D40000C94EC2EEC012B016A016115710519F070
:100D5000FB0191838083C114D10449F0C60102973D
:100D6000839728F020E030E040E050E0DCC0A9901C
:100D70008A2D90E00E943C2F892BC9F7FDE2AF1627
:100D800021F4A9903324339405C08BE2A81609F40A
:100D9000A9903324C114D10421F0E0E1CE16D1048E
:100DA00011F5F0E3AF1669F48881883711F08835C2
:100DB00041F4A980229682E0382A20E1C22ED12C6B
:100DC00012C0C114D10479F4E0E3AE1659F199E9E7
:100DD000E92E99E9F92E99E9092F99E1192F8AE06D
:100DE000C82ED12C3AC0FAE0CF16D10491F080E1A0
:100DF000C816D10429F0E8E0CE16D104F9F415C0E4
:100E0000BFEFEB2EBFEFFB2EBFEF0B2FBFE01B2F73
:100E100024C0A9E9EA2EA9E9FA2EA9E90A2FA9E135
:100E20001A2F1BC0F8E0CF2ED12CEFEFEE2EEFEFF4
:100E3000FE2EEFEF0E2FEFE11E2F0FC0960144277D
:100E400037FD4095542F6FEF7FEF8FEF9FEF0E949C
:100E5000AE2EC901DA017C018D0120E030E040E0D6
:100E600050E060E03601882477FC8094982C70ED87
:100E7000B72EBA0CF9E0FB1570F48A2D81548A3133
:100E800018F499ECB92E06C08A2D81568A3148F59E
:100E900089EAB82EBA0C8B2D90E08C159D050CF5C7
:100EA0006F3FE9F0E216F30604071507B8F0CA0130
:100EB000B901A40193010E947C2E9B01AC018B2DF2
:100EC00090E0A0E0B0E0280F391F4A1F5B1F2817F1
:100ED00039074A075B0710F061E001C06FEFA99086
:100EE000C6CF4114510451F0662311F0219703C07D
:100EF00031FE04C02297F201D183C08330FE07C0C7
:100F000050954095309521953F4F4F4F5F4F67FF6C
:100F10000AC082E290E090934606809345062FEF48
:100F20003FEF4FEF5FEFB901CA01CDB7DEB7E1E1A7
:100F30000C94082FFC0188279927E89421912032EE
:100F4000E9F3293010F02E30C8F32B3241F02D3266
:100F500039F4689404C00E94EF07820F911D21911B
:100F600020532A30C0F31EF4909581959F4F089529
:100F700046E953E00E94BD070895009731F4DA0175
:100F80008D919C91009709F40EC0DC01FB013D910D
:100F90002191222319F03217C9F3FACF332331F408
:100FA000DA011D921C928827992708951197AF9313
:100FB000BF93FB013D912191321771F4332321F44A
:100FC00088279927119702C01E921196FA01A193C2
:100FD000B0839F918F910895222369F7EACF7AE039
:100FE000979F902D879F802D910D112408958091BA
:100FF0009803813019F482E08093980380919803DC
:10100000833019F484E0809398030895E3E0F0E0DE
:1010100089E080935700849190E08670863009F4CF
:1010200091E0892F08951F93182F0E9406088823A6
:1010300079F09FB781E080938D05F894A89588E1B9
:101040008093600010936000112309F0A8959FBF62
:101050001F910895382F20E080911F059091200561
:101060008227932740E061E270E19C01220F331F49
:1010700097FF04C0C9018627972701C0C9014F5FA8
:10108000483099F79093200580931F05089586E3D3
:101090008093BE0380E092ECA1E0B0E08093BF03B8
:1010A0009093C003A093C103B093C20387E08093E1
:1010B000CB0380EC92E9ADEEB9E18093C30390934A
:1010C000C403A093C503B093C60385E08093CC030B
:1010D0008DEE9EEFADEABEED8093C7039093C803FB
:1010E000A093C903B093CA03ADECB3E080E090E0F5
:1010F000863010F0E0E004C0FC01E058FC4FE081D5
:10110000ED9301968831910599F782E08093E5038C
:101110008AE08093E603089580EC91EDA8E9BBE1B5
:1011200080939B0390939C03A0939D03B0939E0395
:1011300010929F031092A0031092A1031092A20399
:1011400008958436910520F4BC0180E090E025C02C
:101150008E3B910550F48A559040BC0180E090E0B0
:101160002AE030E040E050E016C0823D910550F4A6
:10117000845B9040BC0180E090E024E630E040E0F9
:1011800050E009C08D5C9040BC0180E090E028E513
:1011900032E040E050E00E947C2E24E630E040E067
:1011A00050E00E947C2E089590E08C599F4F0E9441
:1011B000A1080895DC019896EC91F0E0E770F070DA
:1011C000E858FC4F808108958F929F92AF92BF9212
:1011D000CF92DF92EF92FF920F931F938C010E94A8
:1011E000DA08D80197962C9130E043E150E0249F33
:1011F000F001259FF00D349FF00D1124EB54FD4FAD
:1012000080809180A280B38090E00F96AA2797FDFE
:10121000A095BA2FBC01CD0120E43FE14DE750E09D
:101220000E947C2EA50194010E94AE2E69017A01D4
:1012300080ED97E0A0E0B0E0C80ED91EEA1EFB1ECC
:10124000D80198968C91887181F060E07EEE8AEBEF
:101250009BE0A50194010E94AE2E28513C4F4F4FB8
:101260005F4FC20ED31EE41EF51E87EE93E0A0E092
:10127000B0E0C80ED91EEA1EFB1EC701B60128EE5B
:1012800033E040E050E00E94AE2ECA01B90128EEE2
:1012900033E040E050E00E947C2E1F910F91FF90C0
:1012A000EF90DF90CF90BF90AF909F908F90089578
:1012B0008F3F910509F010F480E0089522E080301E
:1012C000920710F481E008958050934010F083E07D
:1012D000089582E00895CF92DF92FF920F931F93BB
:1012E000CF93DF93F82FEB016A01182F1695E0E0FA
:1012F00088819981D6018C938A819B8111968C93E8
:1013000011978C819D8112968C9312978E819F816B
:1013100013968C931397288139814A815B816C8164
:101320007D818E819F819295990F990F907C832F5B
:101330008370982B852F8370880F880F982B872FA9
:1013400083708295807F982B14969C9385E090E023
:10135000C80ED91E2896EF5F1E1750F6F0FF21C069
:10136000888199810E945809F82E8A819B810E9468
:101370005809182F8C819D810E945809082F8E8151
:101380009F810E945809F294FF0CFF0C70ECF72229
:101390001295107F1F29182B000F000F012BD6016B
:1013A0000C93DF91CF911F910F91FF90DF90CF9021
:1013B000089523E08032920718F420E030E026C040
:1013C00023E0883E920748F49C012F51334054E0BB
:1013D000369527955A95E1F719C027E0803D920789
:1013E00020F49C012C5D334011C028E0883992071D
:1013F00018F02FEF33E00AC09C01285C374044E02E
:10140000369527954A95E1F72D503C4FC90108952F
:101410009C013695279525753575821B930B9C018C
:101420003695279536952795237333738373937376
:10143000280F391FC901E4E096958795EA95E1F7F1
:10144000820F931F8F709F7021E031E0AC01429FAB
:10145000C001439F900D529F900D1124892F089534
:10146000882339F05F980000289A00005F9A0000F6
:1014700008955F980000289800005F9A0000089582
:101480005F9A000083B15F98000090E09695879581
:10149000817008950F931F93082F5C9A5F985C9852
:1014A00010E0802F80780E94300A000F1F5F1830F4
:1014B000C1F75F981F910F9108958F770E944A0A94
:1014C00008950F931F93082F10E0802F80780E94BB
:1014D000300A000F1F5F1830C1F75F981F910F91FE
:1014E00008950F931F935F9880E000E0182F110F6D
:1014F0000E94400A810F0F5F0830C1F71F910F91C2
:1015000008950E945D0A0E94710A5C9A08951F93D3
:10151000162F80680E944A0A812F0E94610A5C9AF5
:101520001F9108951F931091C7031827EEEBF3E066
:10153000E80FF11D89E767850E94870A8DE3612F17
:101540000E94870A82E4612F0E94870A1F910895F2
:1015500086E20E94810A08950F931F938C018CE10B
:10156000F80164810E94870A8DE1F80165810E947B
:10157000870A8EE1F80166810E94870A80E2F801FD
:1015800067810E94870A81E2F80160850E94870ACC
:1015900082E2F80161850E94870A83E2F801628590
:1015A0000E94870A84E2F80163850E94870A85E227
:1015B000F80164850E94870A8AE2F80165850E9425
:1015C000870A8EE6F80166850E94870A8FE6F80191
:1015D00067850E94870A80E7F80160890E94870A70
:1015E00081E7F80161890E94870A82E7F801628930
:1015F0000E94870A1F910F910895EF92FF920F9317
:101600001F93CF93DF937B018C01603028E3720737
:101610002CE982072CE1920728F520E836E948E911
:1016200050E00E94AE2EE9016897B90180E090E099
:1016300020E839E647E65FEF0E947C2E6E0D7F1DA5
:10164000801F911F32E0660F771F881F991F3A9500
:10165000D1F721E732E040E050E00E94AE2E890150
:1016600080E421C020E03DE241E351E00E94AE2E43
:10167000E9016897B90180E090E020E033ED4EEC9D
:101680005EEF0E947C2E6E0D7F1D801F911F660FE6
:10169000771F881F991F21E732E040E050E00E9449
:1016A000AE2E890180E69E012F71622F680F85E7BB
:1016B0000E94870A86E7612F0E94870A87E7602FCA
:1016C0000E94870ACDB7DEB7E6E00C94132F9F92F5
:1016D000AF92BF92CF92DF920F93DF93CF9300D060
:1016E00000D0CDB7DEB7982E83E00E94810A8093A8
:1016F000E70384E00E94810A8093E80386E060E0CB
:101700000E94870A87E061E00E94870A89E06FE70C
:101710000E94870A8AE065E00E94870A8BE062E106
:101720000E94870A8CE065E10E94870A8DE06DEFD8
:101730000E94870A8EE060E00E94870A992019F0D3
:1017400084E193E008C08091E50323E1829FC0011A
:1017500011248B549D4F0E94AC0A80E36CE80E94D8
:10176000870A82E36FE00E94870A83E362E40E94B3
:10177000870A84E36AE00E94870A85E36AE20E949E
:10178000870A86E36DE20E94870A87E364ED0E9480
:10179000870A88E360E00E94870A89E360E00E948C
:1017A000870A992049F065E7A62E61ECB62E61EC18
:1017B000C62E6EEDD62E08C0A090C703B090C80309
:1017C000C090C903D090CA030AE38D2D9927AA2798
:1017D000BB2789839A83AB83BC83802F69810E9456
:1017E000870A802F8B5F69810E94870ADC2CCB2CB3
:1017F000BA2CAA240F5F0E3341F783E46FEF0E94E7
:10180000870A84E46FEF0E94870A85E46FEF0E94E5
:10181000870A86E46FEF0E94870A992019F08DE607
:1018200066E003C08DE66091CB030E94870A89E7DA
:1018300060E00E94870A8AE76091CC030E94870AD1
:1018400083E760E00E94870A84E760E00E94870ADD
:10185000992029F060EC72E98DEE99E108C0609161
:10186000C3037091C4038091C5039091C6030E9485
:10187000FD0A0F900F900F900F90CF91DF910F9175
:10188000DF90CF90BF90AF909F90089587E061E088
:101890000E94870A8EE764E20E94870A88E063E07C
:1018A0000E94870A88E060E00E94870A87E065E07E
:1018B0000E94870A85E062E00E94870A83E00E9416
:1018C000810A8093E70384E00E94810A8093E80301
:1018D0000895582F40918C04842F90E0FC01EF7004
:1018E000F0709F012F5F3F4F74E0959587957A9533
:1018F000E1F72817390751F0E458FB4F5083842F44
:101900008F5F8F70407F842B80938C0408951F928B
:101910000F920FB60F921124EF92FF920F931F9325
:101920002F933F934F935F936F937F938F939F93E7
:10193000AF93BF93EF93FF93E0909F03F090A003CA
:101940000091A1031091A20389B1A801970120740D
:1019500030704070507090E003E0969587950A953E
:10196000E1F7A0E0B0E081709070A070B07028172F
:1019700039074A075B0709F452C02091840030916F
:10198000850010928500109284008091AD04882318
:1019900009F045C0E5FC02C03695279589E0253C55
:1019A000380708F1809147038630D0F080914703D3
:1019B0008F3FB1F020E00EC0E22FF0E0EE0FFF1FEE
:1019C000DF01A255BB4F8D919C91E95DFC4F918346
:1019D00080832F5F80914703281770F31092AC0427
:1019E000109247031CC082E02D3B3807A8F080917D
:1019F0004703803188F410914703C9010E94D90937
:101A0000E12FF0E0EE0FFF1FE255FB4F9183808343
:101A10001F5F1093470303C08FEF80934703FF912D
:101A2000EF91BF91AF919F918F917F916F915F9156
:101A30004F913F912F911F910F91FF90EF900F9039
:101A40000FBE0F901F90189583E0809380008AE16D
:101A5000809381008FEF9FEF90938900809388009F
:101A600010926F0088E080936D00E8E6F0E08081DE
:101A70008460808308956F3020F086958695805429
:101A800008958DE0689F802D11240895882319F40E
:101A900060E071E002C063E071E083E296E00E94E2
:101AA000302C0895A0E0B0E0E8E5FDE00C94F52EC0
:101AB000182F0E9403299B01AC0180911905909178
:101AC0001A05A0911B05B0911C0569017A01C81A7D
:101AD000D90AEA0AFB0AD701C60189589341A040F6
:101AE000B04010F0109218052093190530931A0594
:101AF00040931B0550931C052091AD04822F81500B
:101B00008230E8F580911805882309F44FC18130AF
:101B100011F482E0BCC1803108F035C1E82FF0E05B
:101B2000E255FB4F10838F5F80931805803109F0D9
:101B3000B0C1A0EBB4E0213039F41196EC911197CB
:101B4000E695E6958C9109C08D919C911197E92FAE
:101B5000E695E695E69596958795E03140F4F0E0B8
:101B600090E0EE0FFF1FE95DFC4F918380831092A0
:101B7000AC04129684E0AE3BB807E9F68AC1233084
:101B800009F004C180911805882321F41F3009F061
:101B900080C10CC1883130F4E82FF0E0E355FB4FF1
:101BA000108374C1883109F0EEC0112309F0EBC035
:101BB000C0E0D0E00BE010E0DE0163E0AA0FBB1F45
:101BC0006A95E1F7C09FB001C19F700DD09F700D65
:101BD0001124FB01E255FB4F80812181922F9770E8
:101BE00095958795FD01EE0FFF1FE95DFC4F9183F1
:101BF0008083FB01E155FB4F308136953695369554
:101C00002181422F4295440F407E842F832B2695BD
:101C100026952695922F977095958795FD01EE0F45
:101C2000FF1FE75DFC4F91838083FB01E055FB4F75
:101C3000808182958695869583704181942F990F36
:101C4000990F292F282B42954695469543708281FE
:101C50008170880F880F382F342B35952795FD011B
:101C6000EE0FFF1FE55DFC4F31832083FB01EE5437
:101C7000FB4F308136952181422F47954427479568
:101C8000842F832B2695922F977095958795FD012C
:101C9000EE0FFF1FE35DFC4F91838083FB01ED544A
:101CA000FB4F308132953F702181422F4295407F1A
:101CB000842F832B22952F70922F9770959587955F
:101CC000FD01EE0FFF1FE15DFC4F91838083FB015F
:101CD000EC54FB4F8081881F8827881F4181942FF7
:101CE000990F292F282B441F4427441F828183707A
:101CF000880F382F342B35952795FD01EE0FFF1FE8
:101D0000EF5CFC4F31832083FB01EA54FB4F3081B1
:101D1000369536952181422F4295440F440F407CE1
:101D2000842F832B26952695922F977095958795CE
:101D3000AA0FBB1FFD01ED5CFC4F918380836954AA
:101D40007B4FFB0120812295269527704181342FFE
:101D5000330F330F330F832F822B942F9295969549
:101D6000977095958795AB5CBC4F11969C938E931D
:101D70002196C230D10509F01FCF8091C40483FDA4
:101D800002C01092AC041092180583C0243009F0F0
:101D900080C040911805442359F4183AB1F41092C8
:101DA000200510921F0588EA0E942A0881E06FC072
:101DB000413019F410931D0504C0423031F41093E2
:101DC0001E05812F0E942A085DC060911E05262FE6
:101DD00030E0220F331FE42FF0E0C90102968E1786
:101DE0009F0734F0433268F7E555FB4F1083E9CF86
:101DF0002D5F3F4F40911F0550912005E217F307DB
:101E000049F4912F80E048275927509320054093AB
:101E10001F0538C0812F90E04817590789F5809138
:101E20001D05813069F5613118F080E180931E0550
:101E3000D0901E054EEAE42E44E0F42E00E010E0BF
:101E40001BC0F701D081C0E0818190E08C2B9D2BDD
:101E500033E0969587953A95E1F70E94D909F80104
:101E6000EE0FFF1FE95DFC4F918380830F5F1F4FD3
:101E700082E090E0E80EF91E0D1518F31092AC0404
:101E80001092180580911805882319F08F5F8093B0
:101E90001805CDB7DEB7E8E00C94112FFF920F9331
:101EA0001F93CF93DF93182F092FF62E8EE30E94F6
:101EB000870A212F302FC901EC0110E005C08FE700
:101EC00069910E94870A1F5F1F15C8F385E064E0CF
:101ED0000E94870A83E00E94810A8093E70384E0DE
:101EE0000E94810A8093E8030E9403296093E9031A
:101EF0007093EA038093EB039093EC0387E069E02F
:101F00000E94870A81E080939803CDB7DEB7E5E0B1
:101F10000C94142F0E944E0F809198038130D9F4B5
:101F20000E9403292091E9033091EA034091EB03D9
:101F30005091EC03621B730B840B950B605A76482F
:101F40008140904040F4E8CF83E296E067E071E0A2
:101F50000E94302C0895809198038130A9F3089550
:101F600083E296E06EE70E94E82D0895A0E0B0E0DD
:101F7000ECEBFFE00C94F42E6C0183E296E06EE74C
:101F80000E94E82D760100E010E0C0E0D0E0B0E271
:101F9000BB2E0AC00830110521F49E012095F601E0
:101FA00020870894E11CF11CF7016081862F8D5772
:101FB000823040F483E296E06DE70E94E82DF7015D
:101FC00060816B2583E296E00E94E82D01151105E2
:101FD00051F0F70180819E01280F311DC32FDD27AD
:101FE000C20FD31FD0700F5F1F4F0930110591F63C
:101FF000CDB7DEB7E9E00C94102FA9E0B0E0E3E044
:10200000F0E10C94FB2E382FE62F8091910490E0A4
:10201000019664E270E00E949B2E982F80939104B9
:1020200088E9898380E18A83913071F0913028F0CA
:10203000923099F09330E1F416C085E08B8381EF04
:102040008C832F5F2D8317C09B8381EF8C8384E665
:10205000489FC00111249D830EC084E08B8381EFD3
:102060008C833D8308C09B8381EF8C83ED8303C009
:102070000E94B00F04C0CE0101960E94B60F2996AF
:10208000E2E00C94172F0F931F93CF93DF93182F39
:10209000092F83E296E06EE70E94E82D212F302F72
:1020A000C901EC0110E000E288818D57823040F4D4
:1020B00083E296E06DE70E94E82D8881802788837F
:1020C00083E296E069910E94E82D1F5F193061F765
:1020D00083E296E06EE70E94E82DDF91CF911F9199
:1020E0000F910895A9E0B0E0E8E7F0E10C94FB2E31
:1020F000382F80919104882379F48EEF89833A8375
:102100006B83842F90E0959587958C832D8319861A
:1021100018861F821E822FC040918C04842F90E06D
:102120009C012F70307054E0959587955A95E1F792
:102130008217930721F18DEF89831A821B82DE01BA
:10214000149620E008C0E458FB4F80818D93405FD7
:102150002F5F263069F0842F90E0FC0134E0F59584
:10216000E7953A95E1F78F709070E817F90759F7FE
:1021700040938C042A83CE0101960E9443108091E3
:10218000910490E0019666E070E00E949B2E80939F
:1021900091042996E2E00C94172F9F92AF92BF9280
:1021A000CF92DF92EF92FF920F931F93B82EA62E3D
:1021B000D42EC22E902E0E9403297B018C01809187
:1021C0007B0420918D0430918E0440918F045091B6
:1021D00090048823B1F0D801C701821B930BA40B94
:1021E000B50B815E9E42A040B04020F12C2DDC1446
:1021F00008F42D2D8B2D6A2D422F292D0E94FD0FC5
:1022000011C0D801C701821B930BA40BB50B8153DE
:102210009547A040B04070F08B2D6A2D4D2D2C2D90
:102220000E947210E0928D04F0928E0400938F044D
:10223000109390041F910F91FF90EF90DF90CF903B
:10224000BF90AF909F90089583E296E06091EE0377
:102250000E94E82D08951F93182F83E296E0612FC6
:102260000E94E82D8091EE0381278093EE031F9159
:1022700008951F93192F0E942B11812F0E942B115B
:102280001F910895DF92EF92FF920F931F93D82E24
:102290007B011092EE0303E216E0C80165EB0E9499
:1022A000E82DC80162E60E94E82D8D2D0E942B11B9
:1022B000C7010E9439111F910F91FF90EF90DF909D
:1022C000089589E060E00E94882988E061E00E942A
:1022D000882987E061E00E94882982E060E00E940E
:1022E000882984E061E00E9488290895892B19F0EB
:1022F0008AE061E002C08AE060E00E94F42908956B
:10230000A0E0B0E0E6E8F1E10C94F32E8CE00E944E
:10231000810A882379F583E296E063E171E00E9407
:10232000302C2D9A80E00E94670B0E94460C2D985D
:1023300021C083E296E00E94AF2D482F8091AD042A
:10234000882321F0842F0E94520D14C0809116051D
:10235000E82FF0E031969F012F7130703197809116
:10236000150590E02817390729F0E451FB4F408309
:102370002093160583E296E00E94752D892BC9F6FD
:1023800080919803843009F08CC00E9403296093E7
:102390009C0470939D0480939E0490939F04611508
:1023A00071058105910561F481E090E0A0E0B0E065
:1023B00080939C0490939D04A0939E04B0939F04EB
:1023C0008091A8049091A90481609093A9048093BE
:1023D000A80483E0809398038FE70E945D0AC3EE10
:1023E000D4E00E94710A899304E0CC3ED007C9F77B
:1023F0004091CE048091E304282F30E0842F90E0B8
:102400008227932786FF40C080E448274093CE046C
:10241000C90188739070C89709F510E014C01F5F58
:102420008091E603E12FF0E084FF06C0ED51FB4F01
:1024300080810E94690C07C0ED51FB4F83E296E05A
:1024400060810E94E82D212F30E08091E30490E02C
:10245000877090708217930714F716C02F7330702F
:10246000232B91F48091E4048093A0048091E504EF
:102470008093A2048091E6048093A3048091E904F0
:102480008093AA041092AB0480911705813019F44F
:1024900082E08093170580911705833011F4109224
:1024A00017050E9403295B016C018091A40490919F
:1024B000A504A091A604B091A7040097A105B105B9
:1024C000C9F0A6019501281B390B4A0B5B0BDA01F9
:1024D000C901885B9B40A040B04060F00E94A80A00
:1024E0008093A1041092A4041092A5041092A60453
:1024F0001092A7048EEB93E00E94E40820919804C8
:102500003091990440919A0450919B048601750181
:10251000E21AF30A040B150BE616F706080719076B
:1025200008F4EAC0A0929804B0929904C0929A0468
:10253000D0929B04A8958091AC04883008F0D4C058
:102540008091AC048F5F8093AC04E0909C04F09089
:102550009D0400919E0410919F04E114F104010573
:10256000110511F18EEB93E00E94E408AE18BF084C
:10257000C00AD10A6A157B058C059D0588F48091F7
:102580009F0384FD04C080ED97E00E9476111092B5
:102590009C0410929D0410929E0410929F0404C00B
:1025A00080E090E00E9476119091CE04907C909310
:1025B000CE0400911605109115050117B1F1809117
:1025C0001705823091F590589093CE048EEB93E0EE
:1025D0000E94DA08893010F048E002C0482F4150CC
:1025E00030E013C03F5FA32FB0E0812F90E0FC01EB
:1025F000E451FB4F2081FD01E253FB4F2083A45F98
:10260000BA4F2C930196182F1F71341710F410171E
:1026100049F710931505832F895C9091CE04892B7F
:102620008093CE0430930C051AC0209117052430F6
:10263000D1F490910C05EDE0F5E0AFECB4E0292F7A
:1026400030E02E0F3F1F02C081918D93E217F307F8
:10265000D9F7995C8091CE04982B9093CE0483E0B7
:102660008093170523C080919304823029F49160F0
:102670009093CE042D9A0FC09093CE042D982223D0
:1026800019F481E08093170580911705833019F4C0
:1026900084E080931705F8948091E603877067E2E1
:1026A00073E04FEC54E00E946B0978942C9A80916F
:1026B00092040E94920A8EEB93E00E94DA08682F3F
:1026C0008EEC94E00E944E0FE0919204EF5FE09355
:1026D0009204E83131F0F0E0E254FC4F8785882322
:1026E00059F41092920408C08091AC04883009F427
:1026F0002D9A89E08093AC048091E603887171F192
:1027000080919803823051F58091A8049091A9049A
:10271000880F991F9093A9048093A80483E0809365
:1027200098030E94460C0E9403296093A4047093AE
:10273000A5048093A6049093A704611571058105F3
:10274000910561F481E090E0A0E0B0E08093A40402
:102750009093A504A093A604B093A7048091E603E8
:1027600084FF1EC08091A8049091A9048E7F0E94CE
:10277000080A182F8091A0046091AA040E943B0DC2
:10278000082F8091A104612F0E943B0D282F80917A
:10279000A2046091A304402F009199030E94CD10E0
:1027A0002C98809193048130C9F0813020F08230E0
:1027B00009F03FC033C08BE00E94272A892BC9F55E
:1027C00081E0809393040E94F528609394047093B1
:1027D000950480939604909397042BC08BE00E94FD
:1027E000272A892B21F50E94F52820919404309105
:1027F00095044091960450919704621B730B840BCF
:10280000950B695E73408040904098F082E0809321
:10281000930480ED97E00E9476110BC08BE00E943C
:10282000272A892B31F080E090E00E9476111092E7
:102830009304CDB7DEB7EAE00C940F2F8AE061E095
:102840000E9488298AE060E00E94F42908951F937D
:10285000182F0E94032960938D0470938E04809337
:102860008F049093900410937B04112329F440E883
:1028700055E260E070E004C040E051EE60E070E0DE
:1028800083E296E00E94EE2C1F910895ACE1B0E047
:10289000ECE4F4E10C94F32E0E9403297B018C01FB
:1028A00081E00E94670BA4E7AA2E6E010894C11C68
:1028B000D11CF3E0BF2EA982C60161E00E948A0FFD
:1028C000B09298030E94460C6AEF70E080E090E0BE
:1028D0000E94292980919803833009F07DC083E20A
:1028E00096E00E94752D892B09F076C00E9403297D
:1028F0006E197F09800B910B6058734C894C914085
:1029000008F06AC0D8CF8FE70E945D0A0E94710A62
:10291000843509F05CC089830E94710A182F00E099
:1029200010937A04009379040E94710A080F111D14
:1029300010937A04009379040E94710A80937804BA
:102940000E94710A80937704813108F040C0FF240F
:1029500007C00E94710A095A1B4FF8018083F39443
:102960000F2D10E08091770490E0880F991F0817D1
:10297000190778F380E78983CE01019661E00E9410
:102980008A0F83E0809398030E94460C62E370E014
:1029900080E090E00E942929809198038330A9F07B
:1029A0008FE70E945D0A0E94710A803581F4898355
:1029B00003EA13E00E94710AF80181938F01F3E0AA
:1029C0000E3B1F07B9F781E003C082E001C083E03E
:1029D0006C96EAE00C940F2F80919803833009F0F5
:1029E00092CFF3CF83E00E94810A8093E70384E0D3
:1029F0000E94810A8093E80387E061E00E94870AD1
:102A00006AE070E080E090E00E9429290E94460C74
:102A1000000008950F931F93082F17C02D9A64E6A6
:102A200070E080E090E00E9429292D9864E670E033
:102A300080E090E00E9429291F5F101778F36CE274
:102A400071E080E090E00E94292910E0F6CF482F45
:102A5000392F25E00DC0F999FECF1FBA842F932F8F
:102A600092BD81BD60BD0FB6F894FA9AF99A0FBE77
:102A7000215059F0F999FECF842F932F92BD81BD3B
:102A8000F89A80B5681739F7089582E00E940A1510
:102A90000895A0E0B0E0EFE4F5E10C94EC2E482EB0
:102AA000562EEE24FF2488249924C0E0D0E0CC24C4
:102AB000DD2436E3332E04C055245394CC24DD2486
:102AC000442069F480919903839DE00111242AE94F
:102AD000E22E23E0F22E99E0892E912C1DC021E0F8
:102AE000421671F480919903839DE00111242B9685
:102AF0008EEBE82E83E0F82E09E2802E912C0CC09C
:102B000032E0431649F419E9E12E13E0F12EB1E069
:102B10008B2E912CC8EDD0E03E016C0C7D1C1092E8
:102B2000200510921F05E3011BC0552059F4F999A7
:102B3000FECFD2BDC1BDF89A80B5F701E00FF11FFD
:102B4000808307C0F701E00FF11FCE0160810E9472
:102B500027150E0D1F1DF80180810E942A0821965D
:102B60009E012619022F10E008151905F0F2CE017A
:102B70005520D9F4F999FECFD2BDC1BDF89A20B540
:102B8000F999FECF2196D2BDC1BD2197F89A80B5A3
:102B900090E0B22EAA248A299B2920911F0530910A
:102BA00020052817390759F487CF21966091200511
:102BB0000E942715CE0160911F050E94271580E015
:102BC00091E0C80ED91E91E0C91693E0D90608F429
:102BD00077CF852DCDB7DEB7E1E10C94082F80E0EB
:102BE00061E00E94491581E061E00E944915089565
:102BF00080E060E00E944915882331F081E060E0C8
:102C00000E944915882331F40E948C080E944708CD
:102C10000E94EF15089582E061E00E944915089531
:102C200082E060E00E94491580919903843020F091
:102C3000109299030E940B1608951F93182F0E945B
:102C4000101680919903811731F0143020F41093FD
:102C500099030E940B161F9108951092550485E662
:102C6000E0EFF3E0DF011D928A95E9F708951F93E5
:102C7000182F8F3711F08830E1F5E0915504EE23DD
:102C800009F455C0E150E0935504F0E0E051FC4FE9
:102C9000108283E296E06DE00E94E82D10E00AC009
:102CA000E12FF0E0E051FC4F83E296E060810E946A
:102CB000E82D1F5F80915504181790F383E296E08A
:102CC00060E20E94E82D83E296E06DE00E94E82D2C
:102CD00010E00AC0E12FF0E0E051FC4F83E296E003
:102CE00060810E94E82D1F5F80915504181790F3B2
:102CF0001CC08B3119F40E942D161FC08D30E9F0D5
:102D00008A30D9F080915504843688F483E296E0C5
:102D1000612F0E94E82D80915504E82FF0E0E051EA
:102D2000FC4F10838F5F8093550480E007C083E2DF
:102D300096E067E00E949C2AF8CF81E01F910895F9
:102D40001F93CF93DF93CDECD3E010E03BC083E241
:102D500096E062E271E00E942D2C83E296E0612F02
:102D60004AE050E00E94AA2B83E296E06FE271E015
:102D70000E942D2C699170E080E090E02091CC03BE
:102D800030E040E050E00E947C2E20E137E240E05D
:102D900050E00E947C2EDC01CB014091C303509196
:102DA000C4036091C5037091C603480F591F6A1F81
:102DB0007B1F83E296E02AE030E00E94712B1F5FC8
:102DC000183119F08881882311F6DF91CF911F9176
:102DD0000895EF92FF920F931F93882339F483E2B3
:102DE00096E066E67AE00E94BA2A3BC090E00E9434
:102DF000A10824E630E040E050E00E94AE2E122F01
:102E0000032FF42EE52E622F732F842F952F2AE0A7
:102E100030E040E050E00E94AE2E83E296E0BA013E
:102E2000A9012AE030E00E94622B83E296E06EE284
:102E30000E949C2A612F702F8F2D9E2D2AE030E05A
:102E400040E050E00E94AE2EAB01BC0183E296E070
:102E50002AE030E00E94622B83E296E063E70E9462
:102E6000CE2A1F910F91FF90EF900895FF920F933C
:102E70001F93CF93DF9383E296E06CE57AE00E94A4
:102E80007B2A8091A303813041F483E296E063E4DE
:102E90007AE00E94BA2AFF2466C0823029F483E2D5
:102EA00096E06CE27AE0F5CF8430A9F783E296E011
:102EB00068E17AE0EECFCF2DD0E0C930D1051CF02B
:102EC0006F2D685C02C06F2D6F5C83E296E00E94FC
:102ED0009C2A83E296E060E17AE00E947B2ABE01B0
:102EE0006F5F7F4F83E296E04AE050E00E94062C3D
:102EF00083E296E065E07AE00E947B2A8E010D5520
:102F00001C4FD8011196EC91E032F8F483E296E080
:102F100068EF79E00E947B2AF8018181803130F0EE
:102F200083E296E063E371E00E942D2CCD55DC4FE7
:102F3000698170E06F7070706F5F7F4F83E296E021
:102F40004AE050E00E94192C0DC0F0E0EF70F070E4
:102F5000EE0FFF1FE85BFC4F6081718183E296E01A
:102F60000E94302CF39480917804F81608F4A3CFD3
:102F700083E296E06DED79E00E947B2A8091BB03AD
:102F80000E94E91683E296E062EC79E00E947B2AD7
:102F90008091BC030E94E91683E296E067EA79E03B
:102FA0000E947B2A8091BD030E94E91683E296E08D
:102FB0006CE879E00E947B2A4091B3035091B403FE
:102FC0006091B5037091B603411551056105710516
:102FD00039F183E296E02AE030E00E94712B83E22F
:102FE00096E069E579E00E947B2A8091B7030E9410
:102FF000D408AB01BC0183E296E02AE030E00E94F5
:10300000712B83E296E065E379E00E947B2A83E2FC
:1030100096E06091B8034AE050E00E94BC2B06C0E5
:1030200083E296E06CE279E00E94BA2A83E296E0BD
:103030006FE079E00E947B2A6091B9037091BA0336
:1030400083E296E04AE050E00E94962B83E296E00D
:1030500062EF78E00E947B2A6091B203603150F405
:1030600070E06F5F7F4F83E296E04AE050E00E949D
:10307000192C06C083E296E069EE78E00E94BA2A35
:1030800083E296E06CEC78E00E947B2A8091B103A9
:1030900080FD03C065E371E002C069E371E083E293
:1030A00096E00E94302C83E296E06FEA78E00E947E
:1030B0007B2A8091B10382700E94460D83E296E0E4
:1030C00060E978E00E947B2A8091B10384700E94BD
:1030D000460D83E296E061E778E00E947B2A8091CA
:1030E000B10388700E94460DCDB7DEB7E5E00C94C1
:1030F000142F1F93CF93DF9383E296E060EB7BE086
:103100000E947B2A4091C3035091C4036091C50380
:103110007091C60383E296E02AE030E00E94712BB2
:1031200083E296E06AE97BE00E947B2A4091C70334
:103130005091C8036091C9037091CA0383E296E07D
:1031400020E130E00E94712B83E296E064E87BE0AE
:103150000E947B2A83E296E06091CB034AE050E034
:103160000E94BC2B83E296E06EE67BE00E947B2A05
:1031700083E296E06091CC034AE050E00E94BC2BD1
:1031800083E296E068E57BE00E947B2ACDECD3E009
:1031900010E012C0112331F083E296E06DE371E09C
:1031A0000E942D2C83E296E069914AE050E00E9453
:1031B000AA2B1F5F183119F08881882359F783E201
:1031C00096E00E94A42A83E296E062E47BE00E94FB
:1031D0007B2A83E296E06091E5034AE050E00E949A
:1031E000BC2B83E296E06DE27BE00E947B2AE091BB
:1031F000E603F0E0E770F070EE0FFF1FE859FC4FB8
:103200006081718183E296E00E94302C83E296E037
:1032100068E17BE00E947B2A8091E60390E0887160
:1032200090708830910589F0893091051CF4892BC4
:1032300039F01BC08031910569F04897B1F40FC097
:1032400083E296E06FE07BE00EC083E296E063E00D
:103250007BE009C083E296E06DEF7AE004C083E290
:1032600096E063EF7AE00E94BA2A83E296E06FED7F
:103270007AE00E947B2A4091BF035091C003609185
:10328000C1037091C20383E296E02AE030E00E941D
:10329000712B83E296E066EC7AE00E947B2A8091B3
:1032A0009F0380710E94460D83E296E06DEA7AE00A
:1032B0000E947B2A80919F0380740E94460D83E2C6
:1032C00096E064E97AE00E947B2A80919F038072F5
:1032D0000E94460D83E296E067E77AE00E947B2A2F
:1032E0008EEB93E00E94E408AB01BC0183E296E020
:1032F0002AE030E00E94622B83E296E062E77AE007
:103300000E947B2A8EEB93E00E94E4089B01AC01B3
:1033100060E472E48FE090E00E94AE2E83E296E0DB
:10332000BA01A9012AE030E00E94622B83E296E014
:103330006FE67AE00E94BA2ADF91CF911F9108953B
:10334000EF92FF920F931F937C0103E216E0C801F6
:103350006F2D70E04AE050E00E94852BC8016EE2BC
:103360000E949C2AB701E4E076956795EA95E1F71B
:103370006F707070C8014AE050E00E94852BC80150
:103380006EE20E949C2A8FE0E822FF24C801B70168
:103390004AE050E00E94852B1F910F91FF90EF9023
:1033A00008950F931F93CF93DF932091EF032F3F47
:1033B000A9F583E296E061EF75E00E947B2A82E640
:1033C00093E00E94A01983E296E060ED75E00E9410
:1033D0007B2A8091790490917A040E94A01983E25B
:1033E00096E06DE975E00E94BA2A83E296E06AE70A
:1033F00075E00E94BA2A83E296E062E675E00E94D8
:10340000BA2A83E296E06DE375E00E94BA2A83E26D
:1034100096E00E94A42A0E94361769C012160CF08A
:1034200066C0332727FD30958091780490E082179D
:1034300093070CF45CC083E296E068E275E00E94BA
:103440007B2A6091EF03772767FD709583E296E012
:103450004AE050E00E94192C83E296E06DEF74E0A0
:103460000E947B2A08E210E03AC0C12FD0E0CC0FC6
:10347000DD1FC95ADB4F288130E08091EF03992787
:1034800087FD909501972817390741F583E296E06B
:103490006FE371E00E942D2C83E296E0602F4AE0FA
:1034A00050E00E94AA2B83E296E063E471E00E9460
:1034B0002D2CE981F0E0EF70F070EE0FFF1FE85B5C
:1034C000FC4F6081718183E296E00E942D2C83E2A3
:1034D00096E067E471E00E942D2C0F5F1F5F8091E2
:1034E0007704181710F283E296E00E94A42ADF9175
:1034F000CF911F910F910895ACE1B0E0E2E8FAE1BD
:103500000C94F52E282F8091EF038F3F09F042C1D4
:10351000822F90E0FC013A97EF36F10508F033C1B5
:10352000EC5CFF4F0C94222F83E296E069E471E09B
:10353000AEC083E296E069E471E00E94302C1CC1C9
:1035400083E296E065E571E00E94302C85E789838F
:10355000DE011296E3EAF3E08BE101900D928150D7
:10356000E1F7CE0101966CE10E948A0F0E94460CA1
:1035700083E08093980368EC70E080E090E00E9424
:10358000292980919803843009F0FDC08FE70E94BB
:103590005D0A0E94710A8983853509F0F4C083E2CF
:1035A00096E06FED74E00E94BA2A83E296E061EC47
:1035B00074E00E94BA2A83E296E063EA74E0ACC049
:1035C00083E296E06DE671E00E94302C89E6898303
:1035D000CE01019661E00E948A0F0E94460C83E0B2
:1035E0008093980368EC70E080E090E00E942929C5
:1035F00080919803843009F0C6C08FE70E945D0A6D
:103600000E94710A89838E010E5F1F4F9DE1E92E92
:10361000F12CEC0EFD1E0E94710AD8018D938D01D4
:10362000AE15BF05C1F7A3EAB3E0FE0132968BE108
:1036300001900D928150E1F78981893409F0A3C08E
:1036400083E296E065E874E00E94BA2A83E296E09D
:1036500067E674E00E94BA2A83E296E069E474E0C7
:103660005BC083E296E067E871E00E94302C8EEF49
:103670008093EF0388C020522750922F905380915F
:103680007804891738F483E296E066E971E00E94D5
:10369000302C79C09093EF036FC084E18093EF03E7
:1036A00083E296E062E174E037C085E18093EF0346
:1036B00083E296E06BED73E02FC086E18093EF0329
:1036C00083E296E064EA73E027C087E18093EF032A
:1036D00083E296E06AE573E01FC088E18093EF0320
:1036E00083E296E069E473E017C089E18093EF0319
:1036F00083E296E065E373E00FC08AE18093EF0315
:1037000083E296E060E273E007C08BE18093EF0311
:1037100083E296E068EF72E00E94BA2A34C083E246
:1037200096E06EED72E00E94BA2A8091B10391E0BA
:103730001DC083E296E068EC72E00E94BA2A809194
:10374000B10392E013C083E296E063EB72E00E9463
:10375000BA2A8091B10394E009C083E296E068E957
:1037600072E00E94BA2A8091B10398E08927809381
:10377000B1038FEF8093EF030E94D11904C083E25D
:1037800096E00E94AF2D83E296E00E94752D892B72
:10379000B1F763C1822F0E943716882309F45DC1F7
:1037A00080915504882321F48FEF8093EF034DC15E
:1037B00080EF93E060E070E040E050E00E949C0603
:1037C0009B01AC016091EF03862F992787FD9095AF
:1037D000A92FB92FFC013197EB31F10508F025C174
:1037E000ED55FF4F0C94222FE62FFF27E7FDF095B4
:1037F0008091780490E08E179F070CF416C1DA01CF
:10380000C9010197A109B1098097A105B10540F04F
:10381000FF2410E008E26F010894C108D10826C017
:10382000ED55FC4F822F81508083E7C0612F70E0FF
:10383000660F771F695A7B4FFB01808190E08C15E2
:103840009D0599F4802F90E0A0E0B0E082179307E7
:10385000A407B50749F4F601ED55FC4FDB011196BD
:103860008C918183FF24F3940F5F1F5F8091770415
:103870001817E0F2C0C02F3F31054105510511F086
:1038800008F0D3C02093BB03B8C02F3F31054105DA
:10389000510511F008F0C9C02093BC03AEC02F3F02
:1038A00031054105510511F008F0BFC02093BD035B
:1038B000A4C08091F0038062803719F581EF93E016
:1038C00060E070E040E050E00E949C069B01AC018B
:1038D000DC01CB010197A109B1090897A105B10548
:1038E00008F0B6C0CA01B90124ED30E340E050E071
:1038F0000E947C2E9B01AC012A5E3C4A4A46554EF2
:1039000024C0863611F581EF93E060E070E040E07E
:1039100050E00E949C069B01AC01DC01CB010197A9
:10392000A109B1090797A105B10508F091C0CA0125
:10393000B90128EA31E640E050E00E947C2E9B016C
:10394000AC01245E3C434E46544E211531054105E1
:10395000510561F0DA01C9018054914EAD49B84179
:103960008158904FAA4FB24008F05FC02093B30334
:103970003093B4034093B5035093B6033EC02F3F3A
:1039800031054105510511F008F04FC02093B703F0
:1039900034C0DA01C9010197A109B1098F3F91052E
:1039A000A105B10508F041C02093B80326C0DA0193
:1039B000C901845C9940A040B0408D549D41A04015
:1039C000B04038F43093BA032093B903FF24F39442
:1039D00001C0FF24211531054105510511F48FEF78
:1039E00007C0213131054105510528F4822F81504E
:1039F0008093B20302C0FF20C1F080915604882357
:103A0000D1F48091C7039091C803A091C903B091EC
:103A1000CA030196A11DB11D8093C7039093C803EB
:103A2000A093C903B093CA0306C083E296E068EA94
:103A300071E00E94302C0E942D168FEF8093EF03CF
:103A400083E296E06AE00E94CE2A0E94D11905C066
:103A500021E030E040E050E07DCF6C96E8E00C944F
:103A6000112F83E296E06CE472E00E94BA2A83E2AE
:103A700096E064E372E00E94BA2A83E296E00E9434
:103A8000752D892B31F083E296E00E94AF2D0E94C4
:103A90007C1A0E944614823019F0833069F405C004
:103AA00083E296E066E172E004C083E296E06FEFA5
:103AB00071E00E94BA2A08958FEF8093EF0310926D
:103AC00056040E94D1190CC083E296E00E94752D25
:103AD000892B31F083E296E00E94AF2D0E947C1A80
:103AE0008091EF038E3F81F708958091EF0399272E
:103AF00087FD9095A92FB92FFC013196EB30F10588
:103B000008F074C0E254FF4F0C94222F83E296E039
:103B100064E678E00E94BA2A82E693E00E94A01947
:103B200083E296E06CE478E00E94BA2A83E296E0B1
:103B300067E278E00E94BA2A83E296E06DEF77E0D0
:103B40000E94BA2A83E296E06CED77E00E94BA2ADE
:103B500083E296E06FEA77E00E94BA2A83E296E079
:103B600069E877E00E94BA2A83E296E065E677E0AA
:103B70000E94BA2A83E296E06EE377E00E94BA2AB6
:103B800083E296E00E94A42A0E9479182FC083E263
:103B900096E061E277E028C083E296E06CEF76E0A1
:103BA00023C083E296E067EE76E01EC083E296E0F3
:103BB00068EC76E019C083E296E064E876E014C031
:103BC00083E296E06FE676E00FC083E296E06AE576
:103BD00076E00E94BA2A83E296E064E176E004C0CF
:103BE00083E296E06EEF75E00E94BA2A6AE070E028
:103BF00080E090E00E94292904C083E296E00E94C0
:103C0000AF2D83E296E00E94752D892BB1F70895C0
:103C1000A2E2B0E0EEE0FEE10C94EB2E8E010F5F2D
:103C20001F4F80E1D8011D928A95E9F783E296E063
:103C300066EC71E00E94302C0E94F21420E431EE18
:103C40004DE958E12F8F38A349A35AA380EC91ED99
:103C5000A8E9BBE18B8F9C8FAD8FBE8F24EF31E045
:103C600040E050E02F8B388F498F5A8F50E5C52E9A
:103C700053ECD52EE12CF12C40E4442E41EE542E91
:103C80004DE9642E48E1742E88249924540133248C
:103C90001E8A1D8A198A1A8A1B8A1C8AFFC083E21F
:103CA00096E00E94AF2D8434B9F0853430F483322D
:103CB000B9F18C3209F0CCC044C0833509F0C8C0DA
:103CC0002F8D38A149A15AA1C901DA012C013D016A
:103CD000882499245401E2C083E296E064E40E94BF
:103CE0009C2A83E296E040E451EE6DE978E12AE017
:103CF00030E00E94D02B83E296E06CE20E949C2A86
:103D000083E296E040EC51ED68E97BE12AE030E0A7
:103D10000E94D02B83E296E06CE20E94CE2ABEC0C5
:103D200019821A821B821C821D821E821F821886A3
:103D300019861A861B861C861D861E861F86188A73
:103D40003AC0339434E0331609F0A8C069817A810F
:103D50008B819C8128EE33E040E050E00E947C2E75
:103D60006F8F78A389A39AA36D817E818F819885B7
:103D70000E947C2E6B8F7C8F8D8F9E8F89859A857C
:103D8000AB85BC858F8B988FA98FBA8F6D857E850B
:103D90008F8598890E947C2E6B017C0190E2C91668
:103DA0009EE4D90690E0E90690E0F90630F48CE153
:103DB00062E30E94870A332471C0A0E3CA16A5E714
:103DC000DA06A0E0EA06A0E0FA0618F48CE162E266
:103DD000F0CFB0E4CB16BCE9DB06B0E0EB06B0E018
:103DE000FB0618F48CE166E2E4CFE0E5CE16E3ECE6
:103DF000DE06E0E0EE06E0E0FE0618F48CE162E1AB
:103E0000D8CFF0E6CF16FAEEDF06F0E0EF06F0E0EE
:103E1000FF0618F48CE165E1CCCF20E7C21621E162
:103E2000D20621E0E20620E0F20618F48CE161E01F
:103E3000C0CF30EAC31636E8D30631E0E30630E0FF
:103E4000F30618F48CE163E0B4CF8CE165E0B1CF08
:103E500030ED232E280E49E0421500F1032D10E02D
:103E6000000F111F000F111F81E090E08C0F9D1FAC
:103E7000080F191FD8016D917D918D919C912AE0B9
:103E800030E040E050E00E947C2E620D711D811DEB
:103E9000911DF801608371838283938383E296E0AE
:103EA0000E94752D892B09F0FACE81149104A1048A
:103EB000B10489F4C301B2010E94FD0A61E070E01F
:103EC00080E090E00E942929FFEFFE8B1D8A198A6D
:103ED0001A8A1B8A1C8A2F89388D498D5A8D821621
:103EE0009306A406B506E0F40E94A80A29893A8937
:103EF0004B895C89280F311D411D511D298B3A8B3F
:103F00004B8B5C8B3D89381708F48D8B4E89841759
:103F100008F48E8B0894811C911CA11CB11C56C006
:103F2000C301B20128EE33E040E050E00E94AE2E23
:103F300083E296E0BA01A9012AE030E00E94622BF8
:103F400083E296E06CE20E949C2A83E296E06D890F
:103F50004AE050E00E94AA2B83E296E06CE20E94C5
:103F60009C2A69897A898B899C89A50194010E9480
:103F7000AE2E83E296E0BA01A9012AE030E00E9469
:103F8000622B83E296E06CE20E949C2A83E296E038
:103F90006E894AE050E00E94AA2B83E296E06CE230
:103FA0000E94CE2A4C0C5D1C6E1C7F1C8B8D9C8D40
:103FB000AD8DBE8D84159505A605B70520F44F8CF3
:103FC00058A069A07AA08824992454012F8D38A183
:103FD00049A15AA1285E33404040504009F05ECFCD
:103FE000A296E2E10C94072FAAE5B0E0EAEFFFE128
:103FF0000C94F72E8B017A018B3009F425C18C309B
:1040000040F5853009F484C0863080F4823009F4AC
:1040100059C0833020F4813009F044C242C083305B
:1040200009F461C0843009F03DC265C0883009F4EC
:104030009DC0893038F4863009F486C0873009F095
:1040400031C28CC0893009F499C08A3009F02AC283
:10405000C9C0893609F476C18A3680F4863609F4F7
:1040600021C1873620F4853609F01CC202C187368B
:1040700009F431C1883609F015C235C18C3609F40E
:10408000B8C18D3638F48A3609F467C18B3609F029
:1040900009C2A3C18D3609F4E0C1873C09F002C210
:1040A000F4C181E069E270E00E9442110EEB13E07E
:1040B000F80181918F010E942B11F3E0073E1F0749
:1040C000B9F7F8C182E06BE170E00E94421103EAA7
:1040D00013E0F80181918F010E942B11F3E00E3B58
:1040E0001F07B9F7E7C183E061E070E00E94421169
:1040F0000E944614DDC184E061E070E00E9442113C
:1041000081E00E942B110E9424110E94081ED4C13C
:104110006091770470E0660F771F85E00E9442117E
:1041200000E010E008C0F801E95AFB4F80810E94CE
:104130002B110F5F1F4F8091770490E0880F991F1C
:104140000817190780F3B6C186E062E070E00E94AC
:10415000421182E693E00E943911ACC187E061E030
:1041600070E00E94421180917804A2C188E061E071
:1041700070E00E944211809199039AC186E689837A
:10418000CE01019661E00E948A0F0E94460C83E0F6
:104190008093980368EC70E080E090E00E94292909
:1041A000809198038430E1F48FE70E945D0A0E94B9
:1041B000710A8983863471F489E060E270E00E94BC
:1041C000421110E00E94710A0E942B111F5F1032F1
:1041D000C9F770C189E061E070E00E944211BBC084
:1041E00089E061C18AE069E070E00E9442111092AA
:1041F0009A0380918D05882351F080919F039091BF
:10420000A003A091A103B091A203806809C080918E
:104210009F039091A003A091A103B091A2038F7777
:1042200080939F039093A003A093A103B093A20354
:104230000AE913E0F80181918F010E942B11F3E04C
:10424000033A1F07B9F736C18BE060E270E00E94C5
:104250004211F89400E010E0F801E95DFC4F808124
:104260000E942B110F5F1F4F00321105A9F77894A0
:1042700021C185E661E070E00E944211093211051A
:1042800009F015C120E030E0F901E254FC4FD701FC
:10429000A20FB31F8C9180832F5F3F4F29323105CE
:1042A00099F759C086E661E070E00E9442110B3137
:1042B000110509F0FCC020E030E0F901ED55FC4F9C
:1042C000D701A20FB31F8C9180832F5F3F4F2B31FB
:1042D000310599F740C087E661E070E00E94421125
:1042E0000E94EF1538C088E661E070E00E9442113C
:1042F00085E78A83DE011396E3EAF3E08BE1019020
:104300000D928150E1F7CE0102966CE10E948A0F76
:104310000E94460C83E08093980360E273E080E0A3
:1043200090E00E94292980919803843009F0BFC051
:104330008FE70E945D0A0E94710A8A83853509F021
:10434000B6C009C089E661E070E00E9442110E9497
:1043500047080E948C0881E0ABC08AE661E070E00B
:104360000E94421189E68E8FCE014E9661E00E9436
:104370008A0F0E94460C83E08093980360E273E00A
:1043800080E090E00E94292980919803843009F010
:104390008EC08FE70E945D0A0E94710A8E8F8E0187
:1043A000015E1F4F6AE3E62EF12CEC0EFD1E0E940B
:1043B000710AF80181938F01EE15FF05C1F7A3EA99
:1043C000B3E0FE017F968BE101900D928150E1F701
:1043D0008E8D893409F06BC0BECF8BE661E070E052
:1043E0000E944211F70180810E941D160E94F8155B
:1043F000B2CF8CE661E070E00E94421100321105FC
:1044000071F487E68AAFDE01DB96F70180E2019066
:104410000D928150E1F7CE01CA9661E205C087E4B2
:104420008AAFCE01CA9661E00E948A0F0E94460CB4
:1044300083E0809398036CE474E080E090E00E9455
:10444000292980919803843091F58FE70E945D0AB5
:104450000E94710A873459F57ECF8DE661E070E0E5
:104460000E9442110930110511F520E030E0F901F8
:10447000E656FC4FD701A20FB31F8C9180832F5FAC
:104480003F4F2930310599F766CF87EC61E070E046
:104490000E94421181E00E942B110E94241110926F
:1044A000ED030AC08AEC61E070E00E94421180E0F6
:1044B0000E942B110E942411C65ADF4FE6E00C9493
:1044C000132FA0E0B0E0E7E6F2E20C94F32E84E0D4
:1044D000A82E06E0B02E15E0C12E01E215E0B4E6EC
:1044E000DB2EA2E0EA2EF3E0FF2EA1C083E296E0ED
:1044F0000E94AF2D982F80938C0580918B0583307F
:1045000021F1843028F4813099F08230B8F409C068
:10451000853009F448C0853020F1863009F087C025
:104520005FC0953B09F083C081E080938B057FC01D
:10453000923609F07AC0E0928B0579C090938A0593
:1045400090938905F0928B0572C090938705109225
:10455000880580918905892780938905A0928B051C
:1045600066C0D92FC0E020918705309188052C2B9B
:104570003D2B3093880520938705809189058927F5
:1045800080938905C0928B052536310508F44FC00C
:104590008CEC61E070E00E94421181E00E942B11DE
:1045A0000E94241142C02091850530918605F901B1
:1045B000EF5DFA4F90838091890589278093890563
:1045C0002F5F3F4F309386052093850580918705A7
:1045D000909188052817390750F1B0928B0527C0B4
:1045E00080918905891759F4609185057091860538
:1045F00080918A0541E255E00E94F41F0DC08BECCA
:1046000062E070E00E94421180918A050E942B11A5
:104610008091EE030E942B11F8018D2D11928A9545
:10462000E9F7109286051092850510928B0583E2BA
:1046300096E00E94752D892B09F058CFCDB7DEB7D3
:10464000EAE00C940F2F81E08093ED0308C083E231
:1046500096E00E94752D892B11F00E9461228091B5
:10466000ED038823A1F70895A0E0B0E0EAE3F3E2C8
:104670000C94F62E0E9403296115710581059105A0
:10468000C9F30E9493061092C7031092C8031092B8
:10469000C9031092CA03DD24E090C703F090C80359
:1046A0000091C9031091CA03102F0F2DFE2CEE2488
:1046B0000E948E062FEF30E040E050E00E94D02EA6
:1046C000E60EF71E081F191FE092C703F092C803F9
:1046D0000093C9031093CA03D39444E0D416E1F6BF
:1046E000CDECD3E000E010E090E1E92E97E2F92E66
:1046F0004EC00F5F19F40E9447084DC00E948E06FD
:1047000022E330E040E050E00E94D02E6F5FEDECFD
:10471000F3E090E004C08191861759F39F5F9117F1
:10472000D0F38091CC0390E08E9D90018F9D300D51
:104730009E9D300D1124862F90E0AC01249FC00176
:10474000259F900D349F900D1124AA2797FDA095C9
:10475000BA2F2091C3033091C4034091C5035091F7
:10476000C603820F931FA41FB51F20919B03309196
:104770009C0340919D0350919E03281739074A07D7
:104780005B0708F4B6CF69931F5F183121F0888169
:10479000882309F0AECFCDB7DEB7E7E00C94122F37
:1047A0001F931091EF031F3F09F0F1C0893409F402
:1047B00067C08A3428F5883309F479C0893368F4EE
:1047C000803309F486C0813308F06FC08B3109F45F
:1047D0004DC0813209F0D5C03DC0813409F49AC082
:1047E000823438F4893309F472C0803409F0C9C0C6
:1047F00031C0823409F4A1C0863409F0C2C052C06D
:10480000823609F49AC0833690F4883579F1893577
:1048100038F4823509F43FC0833509F0B2C01FC0B7
:104820008A3509F4A9C0813609F0ABC073C082375C
:1048300091F1833730F48636A9F1893609F0A1C0A9
:104840001FC0883799F08A3709F496C0833709F07A
:1048500098C005C083E296E069E471E019C00E9447
:10486000EF1583E296E063ED71E006C00E94F81553
:1048700083E296E06DEE71E00E94302C8EEF7FC0F7
:104880000E9447080E948C0883E296E06CE072E088
:104890000E94302C76C00E94342383E296E065E2C9
:1048A00072E0F6CF0E94A0166CC0805368C083E20D
:1048B00096E06CEE71E00E94BA2A9091E603892F8F
:1048C000885F8871977E892B8093E60320C089E0FA
:1048D00056C083E296E069ED71E00E94BA2A8091A9
:1048E0009F039091A003A091A103B091A20320E1A6
:1048F00030E040E050E082279327A427B52780933B
:104900009F039093A003A093A103B093A2031093DD
:10491000EF0337C083E296E063EC71E00E94BA2AAD
:1049200080919F039091A003A091A103B091A20355
:1049300020E430E040E050E012C083E296E062EB19
:1049400071E00E94BA2A80919F039091A003A091E8
:10495000A103B091A20320E230E040E050E08227C2
:104960009327A427B52780939F039093A003A09338
:10497000A103B093A20302C00E94311D8FEF809368
:10498000EF038091EF038E3F09F4DDC0D4C00E9495
:104990003716882309F4D7C080915504882321F461
:1049A0008FEF8093EF03C7C080EF93E060E070E08B
:1049B00040E050E00E949C069B01AC018091EF0317
:1049C000992787FD9095A92FB92FFC013197E930E0
:1049D000F10508F08CC0E753FF4F0C94222FDA0149
:1049E000C9018154914EAD49B8418F57904FAA4F9C
:1049F000B24008F07CC02093C3033093C4034093BB
:104A0000C5035093C6039AC02093C7033093C803CD
:104A10004093C9035093CA0381E0809356048EC02B
:104A2000283031054105510508F061C02093CB03C2
:104A300085C0DA01C9010197A109B1090A97A10549
:104A4000B10508F054C02093CC0378C080EF93E008
:104A50006DE371E00E94B80710E00EC0183130F429
:104A6000E12FF0E0E254FC4F87871F5F80E090E089
:104A70006DE371E00E94B807009759F00E949A0711
:104A8000009761F706C0E12FF0E0E254FC4F178673
:104A90001F5F1831C0F352C0253031054105510563
:104AA00030F52093E5034AC0DA01C9010197A10955
:104AB000B1090697A105B105D0F48091E603887F7E
:104AC000822B8093E6033AC0DA01C9010197A1095C
:104AD000B1098050924CA140B04048F42093BF03EC
:104AE0003093C0034093C1035093C20327C083E2B5
:104AF00096E068EA71E00E94302C13C08091C703F1
:104B00009091C803A091C903B091CA030196A11D59
:104B1000B11D8093C7039093C803A093C903B093BA
:104B2000CA030E942D168FEF8093EF0383E296E075
:104B30006AE00E94CE2A0E94751D05C0809156042D
:104B40008823E1F2EECF1F9108958FEF8093EF035A
:104B5000109256040E94751D0CC083E296E00E94DC
:104B6000752D892B31F083E296E00E94AF2D0E94D3
:104B7000D0238091EF038E3F81F76AE070E080E000
:104B800090E00E94292904C083E296E00E94AF2DA4
:104B900083E296E00E94752D892BB1F70895AAE271
:104BA000B0E0E5EDF5E20C94F02E0E94F5287B01D3
:104BB0008C0181E00E94670B04C083E296E00E94B2
:104BC000AF2D83E296E00E94752D892BB1F72D98C9
:104BD000DD24D39452E6752E42E0842E912C8C0E67
:104BE0009D1E5E010894A11CB11C33E0C32E0E94DF
:104BF000F52820E030E06E197F09800B910B693CAD
:104C000071058105910510F021E030E08D2D90E0D7
:104C100028233923232B99F10E94F5287B018C014D
:104C20002C9A80ED97E00E9476117982D401EEEB08
:104C3000F3E089E201900D928150E1F7C5016AE24B
:104C40000E948A0F2C9880E090E00E947611C0921A
:104C500098030E94460C62E370E080E090E00E94BE
:104C6000292980919803843051F4C09298038FE7EA
:104C70000E945D0A0E94710A823409F4DD248BE0EF
:104C80000E94272A892B49F5DD24D39426C02D9A2A
:104C90002C9A83E296E00E94AF2D8D30910569F049
:104CA0008E3091051CF40A97B1F407C08332910548
:104CB00069F08234910579F40CC083E296E064EAED
:104CC00071E00E94BA2A0E94A52505C00E94081E14
:104CD00002C00E9423232D982C9883E296E00E9424
:104CE000752D892B09F483CFD2CF8F929F92AF92EB
:104CF000BF92CF92DF92EF92FF920F931F938BE0C0
:104D00000E94272A892B09F083C068EC70E080E0BC
:104D100090E00E94292980E090E00E9476110E9494
:104D2000F5285B016C0160ECE62E62E1F62E012DA8
:104D3000112DEA0CFB1C0C1D1D1D06C08BE00E94F2
:104D4000272A892B09F062C00E94F5286E157F057D
:104D50008007910798F38BE00E94272A892B09F09E
:104D600055C080ED97E00E9476110E94F5287B01E6
:104D70008C0199249394882488E496E2A0E0B0E022
:104D8000A80EB91ECA1EDB1E29C0AE14BF04C00681
:104D9000D10638F480ED97E00E9476118824839440
:104DA0001DC00E94F5286E197F09800B910B693C8C
:104DB00071058105910590F00E94F5287B018C0119
:104DC00080E0992009F481E0982E882319F480E08E
:104DD00090E002C080ED97E00E9476118BE00E9487
:104DE000272A892B91F280E090E00E94761188209A
:104DF00049F0809199038F5F83700E941D160E9475
:104E0000F81506C00E9434230E94EF150E94CF259A
:104E10001F910F91FF90EF90DF90CF90BF90AF90D8
:104E20009F908F90089580E067EF77E042E050E038
:104E30000E9430280895EF92FF920F931F9380E015
:104E40000E9413080E9461118DE061E00E94882990
:104E50008CE061E00E9488298BE060E00E94882954
:104E600083E060E00E94882983E061E00E94F429E9
:104E70008EE061E00E9488298EE060E00E94F429C3
:104E80000E941E1483E296E040E052EC61E070E084
:104E90000E94EE2C0E9410160E94F8150E94240D0C
:104EA0008FEF8093AC040E94132778940E94F5281A
:104EB0007B018C018091AC048F3F09F0C7C00E9438
:104EC000F5286E197F09800B910B605D774080405B
:104ED000904008F0BBC0EECF83E296E00E94AF2D79
:104EE00083E296E00E94752D892BB1F783E296E06C
:104EF00062E472E00E942D2C82E693E00E94A019E9
:104F000083E296E069E572E00E942D2C83E296E050
:104F100062E070E04AE050E00E94192C62E370E029
:104F200080E090E00E94292983E296E00E94752D9E
:104F300004970CF183E296E00E94AF2D8234910534
:104F4000D1F483E296E00E94AF2D8E34910599F45E
:104F500083E296E00E94AF2D8434910561F483E2F0
:104F600096E00E94AF2D819731F480E090E00E949E
:104F700076110E94CF254091BF035091C0036091EC
:104F8000C1037091C203DB01CA010197A109B109F4
:104F90000497A105B10568F44093AD04433029F0AE
:104FA00040E052EC61E070E004C040EA56E861E0A5
:104FB00070E083E296E00E94EE2C0E9475262D9808
:104FC00080E090E00E9476110E94240D80E00E9413
:104FD000670B809192040E94920A0E94460C1092E4
:104FE0001505109216051092170510E015C062E322
:104FF00070E080E090E00E94292980ED97E00E9417
:10500000761162E370E080E090E00E94292980E060
:1050100090E00E9476111F5F80919903811738F705
:105020008091E60390E084FF09C020E088719070D1
:10503000489709F421E0822F0E9427148FE00E94F4
:1050400013081F910F91FF90EF90089580ED97E066
:105050000E9476118BE061E00E94F4292D9A40CFE6
:10506000823000F5E82FF0E0EE0FFF1FE257FA4F15
:1050700071836083882319F08130A1F408C0809186
:1050800069008C7F842B80936900E89A0895809151
:105090006900440F551F440F551F837F842B809355
:1050A0006900E99A08951F920F920FB60F9211248A
:1050B0002F933F934F935F936F937F938F939F9320
:1050C000AF93BF93EF93FF9380918E0590918F05DF
:1050D000892B29F0E0918E05F0918F050995FF91BC
:1050E000EF91BF91AF919F918F917F916F915F9160
:1050F0004F913F912F910F900FBE0F901F901895D9
:105100001F920F920FB60F9211242F933F934F933C
:105110005F936F937F938F939F93AF93BF93EF931F
:10512000FF938091900590919105892B29F0E09152
:105130009005F09191050995FF91EF91BF91AF9185
:105140009F918F917F916F915F914F913F912F919F
:105150000F900FBE0F901F9018951F920F920FB6D1
:105160000F9211242F933F938F939F93AF93BF93ED
:105170008091960590919705A0919805B091990519
:1051800030919A050196A11DB11D232F2D5F2D375A
:1051900020F02D570196A11DB11D20939A058093F3
:1051A000960590939705A0939805B09399058091E3
:1051B000920590919305A0919405B0919505019663
:1051C000A11DB11D8093920590939305A093940522
:1051D000B0939505BF91AF919F918F913F912F9182
:1051E0000F900FBE0F901F9018958FB7F8942091D5
:1051F00096053091970540919805509199058FBF7C
:10520000B901CA0108959FB7F89420919205309191
:105210009305409194055091950586B5A89B06C0CD
:105220008F3F21F02F5F3F4F4F4F5F4F9FBF542F56
:10523000432F322F2227280F311D411D511D82E09F
:10524000220F331F441F551F8A95D1F7B901CA0198
:105250000895EF92FF920F931F93CF93DF937B01FB
:105260008C010E940329EB010EC00E9403296C1BD4
:105270007D0B685E7340C8F30894E108F1080109EA
:105280001109C851DC4FE114F1040105110569F75A
:10529000CDB7DEB7E6E00C94132F789484B5826026
:1052A00084BD84B5816084BD85B5826085BD85B5CA
:1052B000816085BDEEE6F0E0808181608083E1E879
:1052C000F0E01082808182608083808181608083B1
:1052D000E0E8F0E0808181608083E1EBF0E08081B4
:1052E00084608083E0EBF0E0808181608083EAE786
:1052F000F0E080818460808380818260808380810F
:10530000816080838081806880831092C1000895CD
:10531000CF93DF93482F50E0CA018850944FFC018F
:1053200034914C51544FFA018491882369F190E0F3
:10533000880F991FFC01EA53F44FA591B491FC0129
:10534000E053F44FC591D491662351F42FB7F894EC
:105350008C91932F909589238C93888189230BC0FE
:10536000623061F42FB7F8948C91932F9095892334
:105370008C938881832B88832FBF06C09FB7F894B6
:105380008C91832B8C939FBFDF91CF9108958330B5
:1053900071F0843028F48130A1F0823021F514C0FE
:1053A0008630B1F08730D1F08430E9F404C08091C8
:1053B00080008F7703C0809180008F7D8093800074
:1053C000089584B58F7702C084B58F7D84BD08951C
:1053D0008091B0008F778093B00008958091B000E5
:1053E0008F7D8093B0000895FF920F931F93F62E48
:1053F000482F50E0CA01845F934FFC012491CA01F9
:105400008850944FFC0114914C51544FFA0104916F
:105410000023C9F0222319F0822F0E94C729E02F10
:10542000F0E0EE0FFF1FE053F44FA591B4919FB74A
:10543000F894FF2021F48C911095812302C08C9167
:10544000812B8C939FBF1F910F91FF9008950F9315
:105450001F93482F50E0CA01845F934FFC012491B1
:10546000CA018850944FFC0104914C51544FFA01E9
:105470001491112319F420E030E015C0222319F013
:10548000822F0E94C729812F90E0880F991F865292
:10549000944FFC01A591B4918C9120E030E08023E1
:1054A00011F021E030E0C9011F910F910895A0E0B3
:1054B000B0E0EDE5FAE20C94F52E7C016B018A0177
:1054C000C0E0D0E00FC0D6016D916D01D701ED9124
:1054D000FC910190F081E02DC7010995C80FD91FFB
:1054E000015010400115110571F7CE01CDB7DEB79F
:1054F000E8E00C94112FEF92FF920F931F93CF933C
:10550000DF937C018B01C0E0D0E0F8010F5F1F4FFB
:105510006491662359F0D701ED91FC910190F081DF
:10552000E02DC7010995C80FD91FEFCFCE01CDB728
:10553000DEB7E6E00C94132FDC01ED91FC910190B5
:10554000F081E02D09950895EF92FF920F931F933C
:105550008C016DE00E949C2A7C01C8016AE00E94D7
:105560009C2A9C012E0D3F1DC9011F910F91FF9098
:10557000EF900895EF92FF920F931F937C010E948A
:105580007B2A8C01C7010E94A42A9C01200F311F95
:10559000C9011F910F91FF90EF900895EF92FF9234
:1055A0000F931F937C010E949C2A8C01C7010E94CB
:1055B000A42A9C01200F311FC9011F910F91FF9058
:1055C000EF900895CF93DF93EC016115710519F405
:1055D00020E030E00FC0DB010D900020E9F71197CB
:1055E000A61BB70BE881F9810280F381E02DAD01A4
:1055F00009959C01C901DF91CF9108954F925F9267
:105600007F928F929F92AF92BF92CF92DF92EF9252
:10561000FF920F931F93DF93CF93CDB7DEB7A19780
:105620000FB6F894DEBF0FBECDBF2C01742ECB0198
:10563000223008F42AE019A231E2C32ED12CCC0E7C
:10564000DD1E822E9924AA24BB24672D752FA50167
:1056500094010E94AE2E79018A01C801B701A5010B
:1056600094010E947C2E472D461B0894C108D10846
:105670004A3010F4405D01C0495CF6014083E114FA
:10568000F1040105110521F07E2C5F2DC801DDCF4D
:10569000C201B6010E94E22AA1960FB6F894DEBFBD
:1056A0000FBECDBFCF91DF911F910F91FF90EF9073
:1056B000DF90CF90BF90AF909F908F907F905F9042
:1056C0004F900895DC012115310541F4ED91FC91D5
:1056D0000190F081E02D642F099508950E94FE2A23
:1056E0000895EF92FF920F931F937C010E94622B0B
:1056F0008C01C7010E94A42A9C01200F311FC901FF
:105700001F910F91FF90EF900895EF92FF920F93EA
:105710001F939A017B0100E010E0B801A7010E94ED
:10572000622B1F910F91FF90EF900895EF92FF92DF
:105730000F931F937C010E94852B8C01C7010E944F
:10574000A42A9C01200F311FC9011F910F91FF90C6
:10575000EF900895EF92FF920F931F939A01E62E18
:10576000FF2400E010E0B801A7010E94622B1F9106
:105770000F91FF90EF900895EF92FF920F931F9378
:105780007C010E94AA2B8C01C7010E94A42A9C01C3
:10579000200F311FC9011F910F91FF90EF900895C5
:1057A000A0E0B0E0E6EDFBE20C94F52EEC016A011E
:1057B0007B012115310541F4E881F9810190F081E7
:1057C000E02D642F09951BC02A303105B1F477FF15
:1057D00013C06DE20E949C2A8C0144275527BA0110
:1057E0004C195D096E097F09CE012AE00E94FE2A4C
:1057F0009C01200F311F04C02AE00E94FE2A9C0158
:10580000C901CDB7DEB7E8E00C94112FEF92FF92FB
:105810000F931F937B019A010027F7FC0095102F2F
:10582000B801A7010E94D02B1F910F91FF90EF901C
:105830000895EF92FF920F931F937C010E94062C14
:105840008C01C7010E94A42A9C01200F311FC901AD
:105850001F910F91FF90EF9008950E94E22A089502
:10586000EF92FF920F931F937C010E942D2C8C01CD
:10587000C7010E94A42A9C01200F311FC9011F915A
:105880000F91FF90EF90089508951F920F920FB619
:105890000F9211242F933F934F938F939F93EF93E6
:1058A000FF938091C00082FD1DC04091C6002091F1
:1058B000DB053091DC052F5F3F4F2F7330708091F7
:1058C000DD059091DE052817390771F0E091DB05C1
:1058D000F091DC05E556FA4F40833093DC052093C8
:1058E000DB0502C08091C600FF91EF919F918F91DF
:1058F0004F913F912F910F900FBE0F901F901895D1
:105900001F920F920FB60F9211242F933F938F93F4
:105910009F93EF93FF9320911F0630912006809173
:105920002106909122062817390731F48091C10091
:105930008F7D8093C10014C0E0912106F091220672
:10594000E152FA4F20818091210690912206019622
:105950008F73907090932206809321062093C60047
:10596000FF91EF919F918F913F912F910F900FBEDB
:105970000F901F901895A0E0B0E0E1ECFCE20C94D1
:10598000F12EFC011382128288EE93E0A0E0B0E0D9
:1059900084839583A683B7838AE893E09183808389
:1059A0007587648757874687318B208B138B028BD3
:1059B000F58AE48AD78AC68AB18EA08E938E828EAB
:1059C0008F85848F8889858F8989868F8A89878F3B
:1059D0008B8980A32096ECE00C940D2FAF92BF92A0
:1059E000DF92EF92FF920F931F93CF93DF93EC011F
:1059F0007A018B01DD24403081EE580780E0680792
:105A000080E0780711F0DD24D39491E0A92EB12C29
:105A1000EC89FD89DD2069F0C50108A002C0880F6E
:105A2000991F0A94E2F7808360E079E08DE390E0CB
:105A300005C0108260E874E88EE190E0A80197014B
:105A40000E94AE2E21503040404050405695479520
:105A50003795279580E12030380720F0DD2011F0C0
:105A6000DD24D6CFE889F9893083EA89FB89208350
:105A700019A2EE89FF89408121E030E0C9010C8C38
:105A800002C0880F991F0A94E2F7482B4083EE89E1
:105A9000FF894081C9010D8C02C0880F991F0A94AB
:105AA000E2F7482B4083EE89FF894081C9010E8CC3
:105AB00002C0880F991F0A94E2F7482B4083EE89B1
:105AC000FF8980810F8C02C0220F331F0A94E2F7F6
:105AD000209528232083DF91CF911F910F91FF9074
:105AE000EF90DF90BF90AF900895DC011C96ED9190
:105AF000FC911D97E05CFF4F219131918081918154
:105B0000281B390B2F733070C901089583E296E08A
:105B10000E94752D892B11F00E94442C0895DC0100
:105B20001C96ED91FC911D97E05CFF4F2081318127
:105B3000E054F040DF01AE5BBF4F8D919C91119717
:105B40002817390719F42FEF3FEF07C08D919C916B
:105B5000E80FF91F8081282F30E0C9010895DC018A
:105B60001C96ED91FC911D97E05CFF4F20813181E7
:105B7000E054F040DF01AE5BBF4F8D919C911197D7
:105B80002817390719F42FEF3FEF10C08D919C9122
:105B90001197E80FF91F20818D919C911197019623
:105BA0008F73907011969C938E9330E0C901089585
:105BB000DC0191968C919197882339F05496ED9160
:105BC000FC915597808186FFF9CF91961C9208959C
:105BD000CF93DF93EC01EE85FF85E05CFF4F2081E2
:105BE0003181E054F0402F5F3F4F2F733070DF0161
:105BF000AE5BBF4F8D919C91119728173907D1F358
:105C0000E05CFF4F80819181E054F040E80FF91F84
:105C10006083EE85FF85E05CFF4F31832083EE8952
:105C2000FF89208181E090E00F8C02C0880F991FCE
:105C30000A94E2F7282B208381E089A3EC89FD896F
:105C400080818064808381E090E0DF91CF9108952E
:105C50008F929F92AF92BF92CF92DF92EF92FF927C
:105C60000F931F9300D000D00F92EDB7FEB731967F
:105C700084E0ADB7BEB711968C9383E0818387E053
:105C8000828385E0838381E0848383E296E06BE90D
:105C900075E04FED55E025EC30E004EC10E0B0ECA1
:105CA000EB2EF12CA1ECCA2ED12CF2ECAF2EB12CA4
:105CB000E6EC8E2E912C0E94BB2C0F900F900F9033
:105CC0000F900F901F910F91FF90EF90DF90CF906A
:105CD000BF90AF909F908F900895CF93DF930E94D5
:105CE0004D290E941B27C6E8DDE20E948011209703
:105CF000E1F30E94862DF9CF629FD001739FF001DE
:105D0000829FE00DF11D649FE00DF11D929FF00D4B
:105D1000839FF00D749FF00D659FF00D9927729F82
:105D2000B00DE11DF91F639FB00DE11DF91FBD010D
:105D3000CF011124089597FB092E07260AD077FD7D
:105D400004D086D006D000201AF4709561957F4F5C
:105D50000895F6F7909581959F4F0895A1E21A2E28
:105D6000AA1BBB1BFD010DC0AA1FBB1FEE1FFF1FFF
:105D7000A217B307E407F50720F0A21BB30BE40B4F
:105D8000F50B661F771F881F991F1A9469F7609596
:105D90007095809590959B01AC01BD01CF01089550
:105DA00097FB092E05260ED057FD04D0D7DF0AD069
:105DB000001C38F450954095309521953F4F4F4F3A
:105DC0005F4F0895F6F790958095709561957F4F98
:105DD0008F4F9F4F08952F923F924F925F926F92F5
:105DE0007F928F929F92AF92BF92CF92DF92EF926B
:105DF000FF920F931F93CF93DF93CDB7DEB7CA1BEC
:105E0000DB0B0FB6F894DEBF0FBECDBF09942A8816
:105E1000398848885F846E847D848C849B84AA84BE
:105E2000B984C884DF80EE80FD800C811B81AA814B
:105E3000B981CE0FD11D0FB6F894DEBF0FBECDBF16
:105E4000ED010895EE0FFF1F0590F491E02D0994E8
:105E5000AA1BBB1B51E107C0AA1FBB1FA617B70790
:105E600010F0A61BB70B881F991F5A95A9F78095AC
:105E70009095BC01CD010895911106C0803219F0B2
:105E800089508550D0F70895992788270895F89468
:025E9000FFCF42
:105E92004E6F005965730054582074696D656F75B3
:105EA2007421006D6F64756C65206C6F636B656443
:105EB2003F00486F70206368616E6E656C20002041
:105EC20040200053004E2F4100386368002C002C04
:105ED200205B005D20280029004E4F5420454E4192
:105EE200424C45440053656E64696E672073657465
:105EF20074696E677320746F2052580A005265737A
:105F0200657474696E672073657474696E67732053
:105F12006F6E2052580A0041626F72746564206588
:105F2200646974730A00696E76616C6964207365D2
:105F32006C656374696F6E000D0A496E76616C69F7
:105F42006420696E707574202D20646973636172B8
:105F52006465642107007363616E6E6572206D6F04
:105F620064650053657474696E6773207361766546
:105F72006420746F20454550524F4D0A0052657699
:105F820065727465642073657474696E67732066E4
:105F9200726F6D20454550524F4D0A004C6F61643F
:105FA200656420666163746F7279206465666175E9
:105FB2006C74730A004B657920616E6420636861BA
:105FC2006E6E656C732072616E646F6D697A656462
:105FD2000A004F70656E4C52536E672054582073FE
:105FE20074617274696E672000206F6E20485720BA
:105FF2000050504D00525353490053444100534303
:106002004C00525844005458440041494E004C42FE
:106012004545500053504B54524D00534255530086
:1060220053554D44004C4C494E440000342B34002F
:106032003800382B340031320031322B3400313603
:106042000001000000C01200001A400AA1204EA563
:10605200001B1E27522C23308025000005400AA178
:10606200204EA50020244EA52C2330004B00000614
:10607200400AD0009D49007B289D492C233000E135
:10608200000005400A4501D7DC03B81E0EBF0023FD
:106092002E48E801008A400A6001555502AD1E20D3
:1060A200000023C88025000005400AA1204EA5005B
:1060B20020244EA52C233000020002000200020020
:1060C20002000200020002000200020002000200BE
:1060D20002000200020002FF610265026A026E0211
:1060E200720276027A027E0284028B02900295028A
:1060F2009B029B029B029B0235019C02A002A20210
:10610200A602A902AE02350100070B0C1011150000
:10611200160A1322312900000000E82D572A752D96
:06612200AF2D8F2DD82DDA
:00000001FF
